:020000040000FA
:020000003628A0
:08000800CE00030ECF008312AD
:100010008B1C0B288B1081010B114F0E8300CE0E11
:100020004E0E09000F398207A929B229B829BE2925
:10003000C429CA29D029D629DC29E229E829EE29B0
:10004000F429A929A929A9290F398207892A902ADF
:10005000902A902A902A902A902A902A902A902AD0
:10006000902A902A902A9A2AA32AAC2A8316FF2340
:10007000900083163F3085003F3087008312FF30A9
:100080008500FF3087008312073099008316003007
:1000900091008316C83081008312013090008316CE
:1000A00000308C00831210308B00203084008001DF
:1000B000840A60300402031C572881018E018F01DD
:1000C0000B118B100B108C01FF30C4008030BF006F
:1000D000C0010230C300A20152226400C408031D03
:1000E00077288030BF00C0010230C300C40AC30BB0
:1000F00091280230C300440FC40A4408163C031C74
:100100008F2803103F0CCC00400CCD000310CC0C0A
:100110004D0CC0024C08031C013EBF029128BF01D8
:10012000C0014008003CC2003F08031C3F0A803C5D
:10013000C10000000F080F3C03189A288F015222BB
:100140002F08BC003508BD002908BB00EF203B0884
:10015000A9003D08B5003C08AF003008BC003608D7
:10016000BD002A08BB00EF203B08AA003D08B600EE
:100170003C08B0003108BC003708BD002B08BB00AC
:10018000EF203B08AB003D08B7003C08B100320847
:10019000BC003808BD002C08BB00EF203B08AC00B9
:1001A0003D08B8003C08B2003308BC003908BD0067
:1001B0002D08BB00EF203B08AD003D08B9003C080E
:1001C000B3003408BC002E08BB003B213B08AE0046
:1001D0003C08B4004408323C031C78226E283B08DB
:1001E00000380319080012203D1D00293F08CA00ED
:1001F0004008CB004A04031D1129BB01BD010800C2
:10020000BD1C05293E08C90023293D1C10294108B1
:10021000CA004208CB003F0840040319BD1411294D
:1002200008003E0801224030CA07003003180130A0
:10023000C9070318C9034A08BC0700300318013076
:10024000C9070318C903C908031908008316280839
:100250008500C90B2929FF3085008312FF308500F6
:100260008316D8308500FF308500831208001220E5
:100270003E08C90023290038031908001220C608C7
:10028000031D48293E08C700C8010230C500C60A40
:10029000C50B62290230C500460FC60A4608163C47
:1002A000031C60290310470CCC00480CCD00031040
:1002B000CC0C4D0CC8024C08031C013EC70262293D
:1002C000C701C8013A196D294808003CCA0047080F
:1002D000031C470A3E02C90071294808CA004708A2
:1002E000C9004908031D78294A08403C03188D2994
:1002F0004A08BC07003003180130C9070318C903B6
:100300003A080539013A031D8C293A154A08C800F4
:100310004908C7000130C60023214608483C03189D
:1003200008003A080539053A031D9A29BB01BA01AC
:10033000C60108003A080639023A031908000430D9
:10034000BA06C60108001220831628088500831209
:1003500008008316FF3085008312FF3085000030CF
:10036000BE000800FC30A800FD3085000130FA29ED
:10037000FC30A800FE3085000230FA29DD30A800EC
:10038000DF3085000330FA29DD30A800FD3085001C
:100390000430FA29DB30A800FB3085000530FA294B
:1003A000DB30A800DF3085000630FA29FA30A800DB
:1003B000FE3085000730FA29FA30A800FB308500AE
:1003C0000830FA29DE30A800DF3085000930FA292C
:1003D000DE30A800FE3085000A30FA29F930A80086
:1003E000FD3085000B30FA29F930A800FB3085007C
:1003F0000C30FA2983169B001C141A088312BE00C5
:100400000800C901CA0CCB0C0318C907C90CCA0CD7
:10041000CB0C0318C907C90CCA0CCB0C0318C907AD
:10042000C90CCA0CCB0C0318C907C90CCA0CCB0CDD
:100430000318C907C90CCA0CCB0C0318C907C90C8F
:10044000CA0CCB0C0318C907C90CCA0CCB0C031877
:10045000C907C90CCA0CCB0C0318C907C90CCA0CB4
:10046000CB0C0318C907C90CCA0CCB0C0318C9075D
:10047000C90CCA0CCB0C0318C907C90CCA0CCB0C8D
:100480000318C907C90CCA0CCB0C0318C907C90C3F
:10049000CA0CCB0C0318C907C90CCA0CCB0C031827
:1004A000C907080007083F3A3F39A300851D2317F5
:1004B000051EA3178122A3002308031D632AA60398
:1004C0000319A401080023082502031D692AA401B9
:1004D0000800230824020319712A0330A700230807
:1004E000A4000A30A600A70B08002408A5000800F5
:1004F000250803190800220203190800C401250871
:10050000882AFF30C40023080F39031D0800103467
:100510002428A901AA01AB01AC01AD01AE0108007C
:100520002308A900B501B514AA01AB01AC01AD01C6
:10053000AE0108000130A9000230AA000930AB006A
:100540000A30AC00B52A0330A9000430AA000530F7
:10055000AB000630AC00B52A0730A9000830AA006D
:100560000B30AB000C30AC00B52AB501B514B601A8
:10057000B614B701B714B801B814AD01AE01080044
:084000000F000F000F000F007C
:02400E00C43FAD
:1042000000004000400040004000400040003000FE
:0A4210004000400030003000400084
:00000001FF
